:100000000C9482070C94C6070C94C6070C94C60780
:100010000C94C6070C94C6070C94C6070C94C6072C
:100020000C94C6070C94C6070C940A130C94DC13AA
:100030000C94C6070C94C6070C94C6070C94C6070C
:100040000C94C6070C94B62C0C94C6070C94C607E7
:100050000C94C6070C94AE220C94C6070C94C607E9
:100060000C94C6070C94C6070C94C6070C94C607DC
:100070000C94C6070C94C6070C94C6070C94C607CC
:100080000C94C6070C94C6070C94C6070C94C607BC
:100090000C94C6070C94C6070C94C6070C94C607AC
:1000A0000C94C6070C94C6070C94C60749146B142D
:1000B00059156B145915B014D314591528153B153F
:1000C00082188218B118B118F41832194B1B4B1B47
:1000D0004B194B1B4C1A4C1A1F1B4B1B4B1B361B33
:1000E000014702477432014702477432012102215D
:1000F0007432012802280001470247743201470286
:10010000477432012002207432012802280001477E
:1001100002477432014702477432011F021F7432D2
:100120000128022800014702477432014702477440
:1001300032011E021E74320128022800000001C094
:1001400002C003C004C005C0018C028C2E004C000C
:100150002900E100358200001E00140004001D008B
:1001600034004D821F001A0015001B00E1042A71A3
:10017000200009001600060050002C722100130018
:10018000170019004F004A0022000A00070005006E
:100190000000E2005000025400002E000000012088
:1001A0004F00025400002D000000E20023000D006B
:1001B0000B000E000000E60024000F0011001000EC
:1001C00052004B002500180008003600510028722C
:1001D00026001C000C0037002F002B712700330075
:1001E0001200387130004E832D0031003400E500DC
:1001F000008200002E004C002900E1003582000042
:100200001E00140004001D0034004D821F001A005F
:1002100016001B00E1042A712000080007000600F8
:1002200050002C7221001500090019004F004A00EF
:10023000220017000A0005000000E20050000254EE
:1002400000002E00000001204F00025400002D008D
:100250000000E20023001C000B0011000000E6007B
:10026000240018000D00100052004B0025000C0067
:100270000E00360051002872260012000F003700D1
:100280002F002B71270013003300387130004E838C
:100290002D0031003400E500008200000100010063
:1002A00001000100010000003A001E0220022202AB
:1002B000010001003B001F02210223020100010096
:1002C0003C002F0226022F00010001003D003002F9
:1002D00027023000010001003E00310235003502E6
:1002E0000000010001000100000001000000010009
:1002F0000100010000000100000001003F00520069
:1003000051002402000001004000240021001E00D2
:10031000010001004100250022001F0037000100FC
:100320004200260023002000270001004300250290
:100330002E0231002E0001004400450001000100A2
:1003400001000000000000000000000000000000AC
:10035000000006200220000000000100000007202D
:100360000320000000000100000000000420000045
:100370000000010000000000052000000000010056
:10038000000000000000000000000100000000006C
:10039000000000000000010000000000000000005C
:1003A000000001000000000000000000000001004B
:1003B000000000000000000000000100000000003C
:1003C000000000000000010000000000000000002C
:1003D000000001000000000000000000000001001B
:1003E0000000000000000000000000000A002530AE
:1003F000313662003A200025303258000A722F63ED
:100400002030313233343536373839414243444570
:10041000460A000A002530325800626F756E636527
:10042000213A20006C6566742073696465206174EC
:100430007461636865640A006C656674207369643E
:1004400065206E6F7420726573706F6E64696E677D
:100450000A00747279696E6720746F207265736523
:1004600074206D637032333031380A005B735D0085
:100470004B6579626F6172642073746172742E0AC5
:10048000005B575D005B535D005B525D005B445D4C
:10049000005B435D0016034500720067006F004477
:1004A000006F007800200045005A00000016034548
:1004B00000720067006F0044006F00780020004564
:1004C000005A0000000403090409028D0005010020
:1004D000A0FA090400000103010100092111010033
:1004E00001223F000705810308000A0904010001F9
:1004F00003010200092111010001224D00070582BC
:100500000308000A09040200010300000009211188
:100510000100012236000705830308000A090403CD
:100520000002030000000921110100012220000740
:1005300005840320000107050403200001090404C9
:100540000001030000000921110100012239000708
:100550000585031000011201100100000008EDFEE6
:10056000071301000102000105010906A1010507A9
:1005700019E029E715002501950875018102050894
:1005800019012905950575019102950175039101E0
:100590000507190029771500250195787501810255
:1005A000C00631FF0974A1010975150025FF9520CA
:1005B000750881020976150025FF952075089102BE
:1005C000C005010980A101850216010026B7001AA5
:1005D00001002AB700751095018100C0050C0901C2
:1005E000A1018503160100269C021A01002A9C0223
:1005F000751095018100C005010902A1010901A141
:1006000000050919012905150025019505750181C8
:100610000295017503810105010930093115812514
:100620007F95027508810609381581257F9501752A
:10063000088106050C0A38021581257F9501750889
:100640008106C0C005010906A101050719E029E7D7
:100650001500250195087501810295017508810134
:100660000508190129059505750191029501750384
:1006700091010507190029FF150025FF950675084A
:100680008100C00A002530325820006B6579626F06
:100690006172645F7265706F72743A20000A00259F
:1006A000303258006B6579626F6172645F73657494
:1006B0005F6C65643A200064656C5F6B65795F62AE
:1006C00069743A2063616E27742064656C3A202552
:1006D0003032580A006164645F6B65795F626974E7
:1006E0003A2063616E2774206164643A20253032B9
:1006F000580A00646F6E652E0A00626F6F676D6145
:10070000676963207363616E3A202E2E2E200029C4
:100710000A002575002F002575005D28002564005E
:100720002000256400200025640020002564007C52
:100730000025303258006D6F7573656B6579205BED
:1007400062746E7C782079207620685D28726570EE
:100750002F61636C293A205B006D6B5F776865657C
:100760006C5F74696D655F746F5F6D6178203D20AB
:1007700025640A006D6B5F776865656C5F6D6178F5
:100780005F7370656564203D2025640A006D6B5FB2
:1007900074696D655F746F5F6D6178203D202564BD
:1007A0000A006D6B5F6D61785F7370656564203DF5
:1007B0002025640A006D6B5F696E74657276616CEA
:1007C000203D2025640A006D6B5F64656C617920B3
:1007D0003D2025640A006D6B5F776865656C5F740A
:1007E000696D655F746F5F6D6178203D2025640AD7
:1007F000006D6B5F776865656C5F6D61785F7370C6
:10080000656564203D2025640A006D6B5F74696D29
:10081000655F746F5F6D6178203D2025640A006D0F
:100820006B5F6D61785F7370656564203D20256442
:100830000A006D6B5F696E74657276616C203D2095
:1008400025640A006D6B5F64656C6179203D20252D
:10085000640A000A00257500363A20776865656CE1
:100860005F74696D655F746F5F6D61783A20000A2F
:1008700000257500353A20776865656C5F6D617895
:100880005F73706565643A20000A00257500343A8C
:100890002074696D655F746F5F6D61783A20000A3E
:1008A00000257500333A206D61785F73706565646B
:1008B0003A20000A00257500323A20696E7465728C
:1008C00076616C286D73293A20000A002575003185
:1008D0003A2064656C6179282A31306D73293A2099
:1008E000000A092D2056616C756573202D0A004D94
:1008F0003E004D25643E20003F0073657420646512
:100900006661756C740A00433E2000776865726505
:100910002064656C74613A20637572736F723D2553
:10092000642C20776865656C3D25640A53656520F5
:10093000687474703A2F2F656E2E77696B697065D5
:100940006469612E6F72672F77696B692F4D6F75C0
:1009500073655F6B6579730A000A092D204D6F7509
:1009600073656B6579202D0A4553432F713A0971E0
:100970007569740A313A0964656C6179282A3130E5
:100980006D73290A323A09696E74657276616C2852
:100990006D73290A333A096D61785F737065656418
:1009A0000A343A0974696D655F746F5F6D61780A26
:1009B000353A09776865656C5F6D61785F7370655E
:1009C00065640A363A09776865656C5F74696D65B8
:1009D0005F746F5F6D61780A0A703A097072696EB0
:1009E000742076616C7565730A643A0973657420C6
:1009F00064656661756C74730A75703A092B310A07
:100A0000646F776E3A092D310A706775703A092B59
:100A100031300A7067646F776E3A092D31300A0AF7
:100A20007370656564203D2064656C7461202A20C4
:100A30006D61785F7370656564202A202872657027
:100A4000656174202F2074696D655F746F5F6D61DF
:100A500078290A003F004D3E2000433E20004C25EF
:100A6000640A000A092D20436F6E736F6C65202D98
:100A70000A4553432F713A09717569740A6D3A0931
:100A80006D6F7573656B65790A000A092D204D61DC
:100A9000676963202D0A643A0964656275670A789C
:100AA0003A096465627567206D61747269780A6BD2
:100AB0003A096465627567206B6579626F6172647B
:100AC0000A6D3A096465627567206D6F7573650A12
:100AD000763A0976657273696F6E0A733A097374B0
:100AE000617475730A633A09636F6E736F6C652086
:100AF0006D6F64650A302D343A096C617965723026
:100B00002D34284631302D4634290A506175733A08
:100B100009626F6F746C6F616465720A653A09658A
:100B20006570726F6D0A6E3A094E4B524F0A7A3AEF
:100B300009736C656570204C454420746573740AB4
:100B4000000A002575002E6E6B726F3A20000A00B5
:100B50002575002E737761705F6261636B736C61E2
:100B600073685F6261636B73706163653A20000A4A
:100B7000002575002E737761705F67726176655F1F
:100B80006573633A20000A002575002E6E6F5F675B
:100B900075693A20000A002575002E737761705F31
:100BA00072616C745F726775693A20000A0025757E
:100BB000002E737761705F6C616C745F6C67756930
:100BC0003A20000A002575002E636170736C6F6314
:100BD0006B5F746F5F636F6E74726F6C3A20000AA4
:100BE000002575002E737761705F636F6E74726F8E
:100BF0006C5F636170736C6F636B3A20000A002551
:100C0000303258006B65796D61705F636F6E666935
:100C1000672E7261773A20000A002575002E6D6FED
:100C20007573653A20000A002575002E6B657962A0
:100C30006F6172643A20000A002575002E6D6174A0
:100C40007269783A20000A002575002E656E61628F
:100C50006C653A20000A00253032580064656275E0
:100C6000675F636F6E6669672E7261773A20000A6C
:100C70000025750064656661756C745F6C617965EB
:100C8000723A20003F004E4B524F3A206F66660A80
:100C9000004E4B524F3A206F6E0A0074696D6572B8
:100CA0005F636F756E743A202530346C580A006BA0
:100CB0006579626F6172645F6E6B726F3A2025585E
:100CC0000A006B6579626F6172645F69646C653A92
:100CD0002025580A006B6579626F6172645F7072DB
:100CE0006F746F636F6C3A2025580A00686F7374D5
:100CF0005F6B6579626F6172645F6C6564732829EC
:100D00003A2025580A000A092D205374617475731E
:100D1000202D0A004743433A20342E392E332041F8
:100D200056522D4C4942433A20312E382E31204123
:100D300056525F415243483A20617672350A004F5D
:100D40005054494F4E533A204C55464120424F4F44
:100D5000544D41474943204D4F5553454B4559202C
:100D600045585452414B455920434F4E534F4C45E3
:100D700020434F4D4D414E44204E4B524F20353174
:100D8000320A004255494C443A20333064623330D1
:100D9000302D6469727479202830373A35373A3308
:100DA00035204A616E2032372032303136290A0030
:100DB0005649443A20307846454544284572676F85
:100DC000446F7820455A29205049443A20307831E0
:100DD000333037284572676F446F7820455A292091
:100DE0005645523A203078303030310A004445536D
:100DF000433A20742E6D2E6B2E206B6579626F61E5
:100E00007264206669726D7761726520666F722008
:100E10004572676F646F780A000A092D2056657263
:100E200073696F6E202D0A000A6D6F7573653A2025
:100E30006F66660A000A6D6F7573653A206F6E0AF9
:100E4000000A6B6579626F6172643A206F66660AA8
:100E5000000A6B6579626F6172643A206F6E0A00F6
:100E60000A6D61747269783A206F66660A000A6DCD
:100E700061747269783A206F6E0A000A646562755F
:100E8000673A206F6E0A000A64656275673A206FE0
:100E900066660A000A0A626F6F746C6F616465723D
:100EA0002E2E2E2000433E20006565636F6E66691E
:100EB000673A0A00536C656570204C4544207465A0
:100EC00073740A0000000000000000000000000130
:100ED0000204060A0F17202C3A4A5D71879DB3C79A
:100EE000DAE9F5FCFFFCF5E9DAC7B39D87715D4AE5
:100EF0003A2C20170F0A060402010000000000002F
:100F00000000000011241FBECFEFDAE0DEBFCDBF2E
:100F100004B603FE24C08091F9019091FA01A091DA
:100F2000FB01B091FC018730904BA740B04BB9F466
:100F30001092F9011092FA011092FB011092FC013B
:100F400014BE84B7877F84BF88E10FB6F89480937E
:100F50006000109260000FBEE0E0FFE3099511E031
:100F6000A0E0B1E0E8E0FDE502C005900D92AA33F3
:100F7000B107D9F711E0AAE3B1E001C01D92A93F82
:100F8000B107E1F70E9442100C94822E0C940000ED
:100F9000FF93EF93E0913A01F0913B01309709F014
:100FA0000995EF91FF910895FC018591803011F032
:100FB000EFDFFBCF0895FF27E0E230E247FF0CC0F0
:100FC000419597FF09C0EDE26095709580959095E9
:100FD000611D711D811D911D27FF02C0219530E308
:100FE00050E2AA27660F771F881F991FAA1FA41710
:100FF00010F0A41B63955A95A9F7AA3008F0A95FD1
:10100000A05DAF93F395611571058105910541F7D9
:10101000ED3211F4EF93F395F21718F43F93F39533
:10102000FBCF8F91B5DFFA95E1F70895E991F9913A
:101030008591803021F0853219F0AADFF9CF08952B
:1010400020E0E89455915532C1F3503311F468947F
:1010500055915A3348F4505390F3220F022E220F29
:10106000220F200D250FF4CF0EF42195899199912F
:10107000533619F3533729F1533559F1BC018827F9
:101080009927E8945C3621F4899199916894559157
:10109000543639F446EF7EF077FF0DC08FEF9FEFA7
:1010A0000AC055374AE039F0583540E121F0523650
:1010B00042E009F00895FF93EF937DDFEF91FF91F8
:1010C000B7CFFF93EF93FC0181918030B9F360DFDC
:1010D000FBCFFF93EF9368DFF1CFDF93CF93CDB7D3
:1010E000DEB72596A3DFCF91DF910895FC01623032
:1010F00021F128F4662349F0613071F036C0643084
:1011000041F108F1653059F130C08281882311F036
:1011100085EE0CC085EE0EC08281882351F085EEED
:101120000E941F1785EE0E94E71783EE0E941F178B
:101130001CC083EE0E94E71718C08281811115C080
:1011400085E291E00895828181110FC08EE091E0E7
:1011500008958281811109C087EF90E0089582810E
:10116000811103C080EE90E0089580E090E0089542
:1011700080E090E008956091BC017091BD01809184
:10118000BE019091BF010E94AD2156985E982598AE
:101190002D9826982E9827982F98823019F0833012
:1011A00021F00895259A2D9A0895269A2E9A089549
:1011B0008BEB98E0892B11F00E94BB0880E090E057
:1011C000089556985E9825982D9826982E982798D9
:1011D0002F988FEF90E090938900809388009093F0
:1011E0008B0080938A0090938D0080938C00259AC9
:1011F0002D9A2FEF80E792E0215080409040E1F758
:1012000000C00000269A2E9A2FEF80E792E021502E
:1012100080409040E1F700C00000279A2F9A2FEFFE
:1012200080E792E0215080409040E1F700C000004C
:1012300025982D982FEF80E792E021508040904034
:10124000E1F700C0000026982E982FEF80E792E08B
:10125000215080409040E1F700C0000027982F986F
:1012600056985E9825982D9826982E9827982F980E
:10127000089589EA8093800089E080938100249812
:101280002C983F988AB18F748AB96E98479A8BB11F
:10129000806B8BB9769A0E94E10888EB98E0892BE5
:1012A00011F00E94B80880E090E0089580E28093F9
:1012B000000180913C0181110EC00E94A50981E0CE
:1012C00080933C012FEF83ED90E3215080409040CC
:1012D000E1F700C0000080E40E94AB0980930001A8
:1012E00081112EC00E94D50980930001811128C070
:1012F0000E94D50980930001811122C08FE30E94D2
:10130000D5098093000181111BC00E94CD0980E4A2
:101310000E94AB0980930001811112C08CE00E94F1
:10132000D5098093000181110BC00E94D5098093DB
:101330000001811105C08FE30E94D509809300014F
:101340000E94CD098091000108951092B9008AE0B1
:101350008093B800089594EA9093BC009091BC00EB
:1013600097FFFCCF9091B900987F983021F0903191
:1013700011F081E008958093BB0084E88093BC0065
:101380008091BC0087FFFCCF8091B900887F8831B5
:1013900011F0803471F780E0089584E98093BC00F7
:1013A0008091BC0084FDFCCF08958093BB0084E84D
:1013B0008093BC008091BC0087FFFCCF9091B90066
:1013C000987F81E0983209F480E0089584E8809362
:1013D000BC008091BC0087FFFCCF8091BB000895CA
:1013E00080910001811115C080E40E94AB098093B7
:1013F000000181110CC082E10E94D5098093000197
:10140000811105C08FEF0E94D509809300010E94D1
:10141000CD0984B1807F84B985B1807F85B98AB1D7
:10142000837F8AB98BB1837F8BB93E9846980895A4
:101430000E945609809300010E94F00980B38C70CD
:1014400080BB81B3836F81BBAEE3B1E0ECE4F1E03C
:101450008EE08E0F11921D928E13FCCF89E399E0DE
:10146000892B11F00C94390908959F92AF92BF9285
:10147000CF92DF92EF92FF920F931F93CF93DF9360
:10148000809100018823E1F080913D018F5F80937E
:101490003D01811115C082E594E00E94D4070E94AD
:1014A000560980930001882329F088E394E00E9484
:1014B000D40706C084E294E00E94D4070E94E108A9
:1014C0000EE311E0C0E0D0E0BB24B39482E0A82E8C
:1014D000CC24C394D12C25E1E22E24E0F22EC73097
:1014E000D10500F580910001811164C080E40E9463
:1014F000AB0980930001811112C082E10E94D509DD
:101500008093000181110BC0C6010C2E01C0880F11
:101510000A94EAF780950E94D509809300010E9401
:10152000CD0948C0CA30A1F028F4C83059F0C930FC
:1015300061F005C0CC3089F070F0CD3089F0209A90
:10154000289810C0219A29980DC0229A2A980AC07A
:10155000239A2B9807C0529A01C0539A5B9802C0F5
:101560003E9A469890EA9A95F1F79FB1799902C010
:1015700082E001C080E091709B25982B7C9902C08D
:1015800084E001C080E0892B7D9902C038E001C071
:1015900030E0832B7E9902C020E101C020E0822B45
:1015A0009FB19095991F9927991F9295990F907EB9
:1015B000892B10C080910001811174C080E40E94C9
:1015C000AB0980930001882309F459C0912C0E9433
:1015D000CD09892DF8019081981739F18083809188
:1015E0000101882301F18091D70180FF04C08AE1C5
:1015F00094E00E94D4078091D70180FF0CC08091B5
:1016000001011F928F93FF92EF920E946D080F903D
:101610000F900F900F908091D70180FF04C083E15D
:1016200094E00E94D407A09201010E94F009219643
:101630000F5F1F4FCE30D10509F051CF80910101CE
:101640008823B1F0815080930101882339F08FE91C
:101650009FE00197F1F700C000000AC0ACE4B1E0E0
:10166000EEE3F1E0CF01825F91919D938E13FCCF69
:1016700088ED98E0892BC1F00E94D80815C083E15D
:101680000E94D509809300018111A0CF81E40E94BE
:10169000AB0980930001811199CF0E94E609982E31
:1016A000909495CF80E096CF81E0DF91CF911F910C
:1016B0000F91FF90EF90DF90CF90BF90AF909F90F1
:1016C0000895E82FF0E0E45BFE4F80810895CF920B
:1016D000DF92EF92FF920F931F93CF93DF938CEFE4
:1016E00093E00E94D4078CE4E82E81E0F82EC0E05D
:1016F000D0E097EFC92E93E0D92E0EEE13E0DF93E2
:10170000CF93DF92CF920E946D0884EF93E00E9406
:10171000D407F70181917F0190E00E9413229F93EB
:101720008F931F930F930E946D088CEE93E00E949D
:10173000D40721968DB79EB708960FB6F8949EBF32
:101740000FBE8DBFCE30D105D1F6DF91CF911F9165
:101750000F91FF90EF90DF90CF9008958B3B910514
:1017600078F4883A910540F5853A9105D0F48430B3
:10177000910508F0B1C08130910509F4ADC06BC08E
:10178000803E910508F467C0883E910508F4A4C026
:101790009C01205F31092031310508F05CC0906563
:1017A0000895853A910509F459C0863A910509F0E2
:1017B00058C082E890E40895883A910509F454C02D
:1017C000893A910509F453C08A3A910509F452C047
:1017D0008B3A910509F451C08C3A910509F450C037
:1017E0008D3A910509F44FC0803B910509F44EC034
:1017F0008E3A910509F44DC08F3A910509F44CC019
:10180000813B910509F44BC0823B910509F44AC024
:10181000833B910509F449C0843B910509F448C014
:10182000853B910509F447C0863B910509F446C004
:10183000873B910509F445C0883B910509F444C0F4
:10184000893B910509F443C08A3B910509F442C0E4
:1018500080E094E4089580E090E0089581E890E4C9
:10186000089583E890E4089582EE94E4089589EE63
:1018700094E408958AEE94E4089585EB94E4089541
:1018800086EB94E4089587EB94E408958CEC94E45B
:1018900008958DEC94E4089583E895E408958AE82A
:1018A00095E4089582E995E4089584E995E408951E
:1018B00081E296E4089583E296E4089584E296E452
:1018C000089585E296E4089586E296E4089587E215
:1018D00096E408958AE296E40895089596E0799F43
:1018E000F001112494E5899FE00DF11D1124E60F0C
:1018F000F11DEE0FFF1FE45BFE4F8591949108955B
:10190000880F991FFC01E454F0408591949108954B
:10191000880F991FFC01E45CFE4F85919491089516
:1019200026E0729FF001112444E5849FE00DF11D33
:101930001124E60FF11DEE0FFF1FE45BFE4F8591B2
:1019400094919C013A9521154FE1340708F41AC18E
:101950003F512115304120F49F700E94880C08955A
:101960009C0130532115304118F49927906C08954B
:10197000811520E5920769F40E946D1B4FEF84E307
:101980009CE0415080409040E1F700C000000C9482
:10199000D322813020E5920731F48091D701816014
:1019A0008093D70108959C0130552115304108F0EE
:1019B00051C0292F33272F70332721303105D9F417
:1019C000AC014370552702C0220F331F4A95E2F73E
:1019D0003C68AC0164E0440F551F6A95E1F7442769
:1019E0005370242B352B73E0880F991F7A95E1F7FC
:1019F000807699271DC02230310529F4982F882739
:101A0000816F906A089523303105A9F4AC014370C9
:101A1000552721E030E002C0220F331F4A95E2F73C
:101A20003C6843E0880F991F4A95E1F7807E9770E4
:101A3000822B932B089524303105E1F4AC014370DF
:101A4000552721E030E002C0220F331F4A95E2F70C
:101A50003A68E7CF9C0130572115304118F49F7048
:101A6000906208959C0130582115304118F49F7000
:101A7000906A0895803E9105E0F4803C910558F508
:101A80008133910509F46FC048F48932910509F456
:101A900063C08A32910509F46DC072C08933910523
:101AA000E9F082389105D1F08533910509F44DC0F4
:101AB00067C0833E910581F138F4803E9105B9F00D
:101AC000823E9105D9F05CC0863E910561F1873E6A
:101AD0009105A1F155C00E94800C08952091EA0162
:101AE00020FD02C021FF4CC080EE90E049C08091F3
:101AF000EA0180FFF9CF89E390E042C08091EA01DA
:101B000082FF0EC08091EA0184FF03C080E090E074
:101B100037C083EE90E034C08091EA0182FFF2CFBB
:101B200082EE90E02DC08091EA0183FF0BC080918E
:101B3000EA0184FDEBCF87EE90E022C08091EA01BC
:101B400083FFF5CF86EE90E01BC08091EA0185FF10
:101B500007C089E290E014C08091EA0185FFF9CFC7
:101B600085E390E00DC08091EA0186FF07C08AE21C
:101B700090E006C08091EA0186FFF9CF81E390E012
:101B80000E94AE0B0895089580916D0108959FB74E
:101B9000F89410925C019FBF9091F001943009F08D
:101BA00057C09091E9009F703091EC00232F217075
:101BB00030FD20E8922B24E02093E9002091EB00F7
:101BC00020FF43C02091EE0027FF3FC020915A0123
:101BD000222321F02091E80025FF37C010925A01FE
:101BE00026E03091E80035FD15C03091F001343029
:101BF00061F53091EB0035FD28C0215021F481E0E2
:101C000080935A0122C0EFE9FFE03197F1F700C05D
:101C10000000E7CF8093F1008091E80085FD0AC0C5
:101C20008091E80080FFFCCF8091E8008E77809360
:101C3000E80006C08FB7F89421E020935C018FBFC5
:101C40009F709093E90080E008959F709093E90061
:101C50008FEF0895CF93DF9300D01F92CDB7DEB7FB
:101C60009C018091F001843019F593E099833B83C6
:101C70002A839093E9008FEF9091E800815095FDC1
:101C800006C095ED9A95F1F700008111F5CF80918E
:101C9000E80085FF0DC040E050E063E070E0CE0159
:101CA00001960E94FA108091E8008E778093E800F8
:101CB0000F900F900F90DF91CF910895CF93DF9306
:101CC00000D01F92CDB7DEB72091F001243021F56E
:101CD00022E029839B838A8383E08093E9008FEF4E
:101CE0009091E800815095FD06C095ED9A95F1F729
:101CF00000008111F5CF8091E80085FF0DC040E024
:101D000050E063E070E0CE0101960E94FA108091ED
:101D1000E8008E778093E8000F900F900F90DF918E
:101D2000CF9108952091F0012430F1F422E0209326
:101D3000E9002FEF3091E800215035FD06C035ED68
:101D40003A95F1F700002111F5CF2091E80025FF29
:101D50000BC040E050E065E070E00E94FA10809116
:101D6000E8008E778093E8000895CF93DF93209169
:101D7000F001243009F048C0EC0180910C01882367
:101D8000E1F080910D018823C1F085E08093E900A6
:101D90008FEF9091E800815095FD06C095E19A95EE
:101DA000F1F700008111F5CF8091E80085FF2CC08C
:101DB00040E050E060E170E017C081E08093E9000E
:101DC0008FEF9091E800815095FD06C095ED9A95B2
:101DD000F1F700008111F5CF8091E80085FF14C074
:101DE00040E050E068E070E0CE010E94FA1080917F
:101DF000E8008E778093E80080E1FE01ADE5B1E078
:101E000001900D928A95E1F7DF91CF91089581E9D4
:101E100094E00E94D4078091EF01811109C00E94D3
:101E20008F120E94EC128091E20084608093E200A5
:101E300008958DE894E00E94D4071092EF01089570
:101E400089E894E00C94D40785E894E00E94D407D4
:101E50000C94A32C81E894E00E94D4070E9469228C
:101E60000E94A92C0E9491150C94C30D20915B0136
:101E70002F5F822F62E30E94172E992319F020937F
:101E80005B01089510925B0180915C01882371F1E0
:101E90008091F001843041F58091E9008F702091AC
:101EA000EC00922F917020FD90E8892B94E09093A4
:101EB000E9009091EB0090FF14C09091EE0097FF25
:101EC00010C09091E80095FF03C01092F100F9CF87
:101ED0009091E80090FF05C09091E8009E77909364
:101EE000E8008F708093E90010925C01089542E051
:101EF00061EC81E00E94091242E061EC82E00E9404
:101F0000091242E061EC83E00E94091242E261ECB6
:101F100084E00E94091242E161EC85E00C94091210
:101F20008091F201833009F455C030F4813071F0B2
:101F3000823009F48EC008958A3009F47AC08B305B
:101F400009F460C0893009F09CC020C08091F10183
:101F5000813A09F096C08091E800877F8093E8007D
:101F60008091F5019091F601892B21F460E18DE5D6
:101F700091E003C060E080E090E070E00E944511D5
:101F80008091E8008B778093E80008958091F101BB
:101F9000813209F076C08091F5019091F6010097A9
:101FA00019F0049709F06DC08091E800877F809355
:101FB000E8008091E80082FD05C08091F001811168
:101FC000F8CF5FC08091F10080936D018091E800AF
:101FD0008B7753C08091F101813A09F052C0809112
:101FE000F5019091F601892B09F04BC08091E80032
:101FF000877F8093E8008091E80080FFFCCF80918C
:102000000C0136C08091F1018132D9F58091F50142
:102010009091F601892BA9F58091E800877F809344
:10202000E8000E943E128091F30180930C010C9411
:102030006D1B8091F101813221F58091E800877F4D
:102040008093E8000E943E128091F40180936E011B
:1020500008958091F101813AA1F48091E800877F91
:102060008093E8008091E80080FFFCCF80916E01B2
:102070008093F1008091E8008E778093E8000C94C3
:102080003E12089584B7877F84BF88E10FB6F89425
:1020900080936000109260000FBE90E080E80FB661
:1020A000F89480936100909361000FBE0E941E1609
:1020B0000E948F120E94EC128091E2008460809353
:1020C000E20087EC9DE00E94A82178940E9471159F
:1020D0000E94201682E091E00E948C150E94912CB3
:1020E00080E794E00E94D4078091F001853089F464
:1020F0008CE694E00E94D4070E942D228091EE018C
:10210000882391F30E945522882371F30E94E410E2
:10211000EBCF0E944E16E8CF292F3327233031050D
:10212000C9F064F42130310581F02230310509F025
:1021300043C08DE890E029EC34E042C02132310503
:10214000F1F02232310541F137C082E190E026E51D
:1021500035E036C099278130910541F082309105F4
:1021600041F0892B49F5E5ECF4E005C0EDEAF4E037
:1021700002C0E5E9F4E0849190E09F0121C0653060
:10218000D8F4E62FF0E0EE0FFF1FEB5DFE4F20814D
:10219000318189E090E014C0653070F470E0FB019B
:1021A000EE0FFF1FE55EFE4F20813181FB01EA5EED
:1021B000FE4F808190E004C080E090E020E030E0BD
:1021C000FA0131832083089580E189BD82E189BDD0
:1021D00009B400FEFDCF8091D8008F7D8093D80098
:1021E0008091E00082608093E0008091E00081FDBA
:1021F000FCCF0895CF92DF92EF92FF920F931F933F
:10220000CF93DF93EC018B016A010E945D12811173
:1022100033C0C114D10439F0F60180819181081BCB
:10222000190BC80FD91FE12CF12C0115110519F15B
:102230008091E80085FD16C08091E8008E7780933C
:10224000E800C114D10449F0F60180819181E80EC3
:10225000F91EF182E08285E00FC00E945D128823A2
:1022600021F30AC089918093F10001501109FFEF19
:10227000EF1AFF0ADACF80E0DF91CF911F910F9123
:10228000FF90EF90DF90CF9008952091F70130916B
:10229000F8012617370748F06115710539F42091C8
:1022A000E8002E772093E80001C0B90140E06115F5
:1022B0007105A9F12091F001222309F443C02530D2
:1022C00009F442C02091E80023FD40C02091E800BD
:1022D00022FD32C02091E80020FFE9CF4091F300B9
:1022E0002091F20030E0342BFC01CF016115710523
:1022F00059F02830310540F481918093F10061500C
:1023000071092F5F3F4FF1CF41E02830310509F0CF
:1023100040E02091E8002E772093E800C8CF4111DB
:10232000C9CF0AC08091F001882361F0853061F047
:102330008091E80083FD0AC08091E80082FFF2CF1F
:1023400080E0089582E0089583E0089581E0089593
:102350002091F7013091F8012617370748F06115F1
:10236000710539F42091E8002E772093E80001C030
:10237000B901FC0120E06115710591F18091F00136
:10238000882309F440C0853009F43FC08091E800FB
:1023900083FD3DC08091E80082FD2FC08091E80060
:1023A00080FFE9CF2091F3008091F20090E0922B22
:1023B0006115710559F08830910540F424912093FE
:1023C000F1003196615071090196F2CF21E0089732
:1023D00009F020E08091E8008E778093E800CBCF71
:1023E0002111CCCF0AC08091F001882361F08530A3
:1023F00061F08091E80083FD0AC08091E80082FFCF
:10240000F2CF80E0089582E0089583E0089581E0AE
:102410000895982F973058F59093E900981739F060
:102420007091EC002091ED005091F00003C0242F3A
:10243000762F50E021FF19C03091EB003E7F3093A2
:10244000EB003091ED003D7F3093ED003091EB00DB
:1024500031603093EB007093EC002093ED005093CB
:10246000F0002091EE0027FF07C09F5FD3CF8F7051
:102470008093E90081E0089580E008958091F10162
:1024800087FF11C08091E80082FD05C08091F001B6
:102490008111F8CF11C08091E8008B770BC080913B
:1024A000F001882349F08091E80080FFF8CF809107
:1024B000E8008E778093E80008952091E400309141
:1024C000E50095E64091EC00842F817040FF22C02A
:1024D0008091E80080FD1CC08091F001882391F07C
:1024E000853091F08091EB0085FD10C04091E400B3
:1024F0005091E5004217530729F39A01915011F7C3
:1025000084E0089582E0089583E0089581E00895CD
:1025100080E008954091E80042FFDECF08950E94D8
:10252000FD120E940513E0EEF0E08081816080835F
:10253000E8EDF0E080818F77808319BCA7EDB0E0F3
:102540008C918E7F8C9380818F7E80831092EF019F
:1025500008950F931F93CF93DF930E94FD120E9463
:102560000513C8EDD0E088818F77888388818068E3
:10257000888388818F7D888319BC1092F001109226
:10258000EC011092EE011092ED0100EE10E0F80166
:1025900080818B7F808388818160888342E060E0D6
:1025A00080E00E940912E1EEF0E080818E7F80835E
:1025B000E2EEF0E0808181608083808188608083AA
:1025C000F80180818E7F8083888180618883DF919C
:1025D000CF911F910F910895E8EDF0E080818F7EFB
:1025E0008083E7EDF0E080818160808384E082BFBA
:1025F00081E08093EF010C94A912E8EDF0E0808176
:102600008E7F80831092E20008951092DA0010927B
:10261000E10008951F920F920FB60F9211242F938D
:102620003F934F935F936F937F938F939F93AF935A
:10263000BF93EF93FF938091E10082FF0BC08091E5
:10264000E20082FF07C08091E1008B7F8093E10070
:102650000E94360F8091DA0080FF1FC08091D80061
:1026600080FF1BC08091DA008E7F8093DA0080911A
:10267000D90080FF0DC080E189BD82E189BD09B428
:1026800000FEFDCF81E08093F0010E94070F05C09E
:1026900019BC1092F0010E94190F8091E10080FF97
:1026A00019C08091E20080FF15C08091E2008E7F0A
:1026B0008093E2008091E20080618093E20080914B
:1026C000D80080628093D80019BC85E08093F00127
:1026D0000E94240F8091E10084FF30C08091E200CD
:1026E00084FF2CC080E189BD82E189BD09B400FE70
:1026F000FDCF8091D8008F7D8093D8008091E1003C
:102700008F7E8093E1008091E2008F7E8093E200D3
:102710008091E20081608093E2008091EC01882347
:1027200011F084E007C08091E30087FD02C081E0E2
:1027300001C083E08093F0010E942A0F8091E100A4
:1027400083FF29C08091E20083FF25C08091E100D2
:10275000877F8093E10082E08093F0011092EC018A
:102760008091E1008E7F8093E1008091E2008E7F76
:102770008093E2008091E20080618093E20042E079
:1027800060E080E00E9409128091F00088608093F0
:10279000F0000E94200FFF91EF91BF91AF919F91A8
:1027A0008F917F916F915F914F913F912F910F90FA
:1027B0000FBE0F901F9018951F920F920FB60F9299
:1027C00011242F933F934F935F936F937F938F9336
:1027D0009F93AF93BF93CF93DF93EF93FF93C091FA
:1027E000E900CF708091EC00D82FD17080FDD0E847
:1027F0001092E9008091F000877F8093F000789438
:102800000E9420141092E9008091F000886080936B
:10281000F000CD2BCF70C093E900FF91EF91DF91D5
:10282000CF91BF91AF919F918F917F916F915F9168
:102830004F913F912F910F900FBE0F901F901895C1
:102840001F93CF93DF93CDB7DEB7AA970FB6F89457
:10285000DEBF0FBECDBFE1EFF1E088E08E0F9091BB
:10286000F10091938E13FBCF0E94900F8091E800AE
:1028700083FF1FC18091F1019091F201492F50E037
:102880004A30510508F015C1FA01EA5AFF4F0C947D
:10289000372E803881F0823809F00BC18091F50124
:1028A0008F708093E9008091EB0085FB882780F989
:1028B0001092E90006C08091ED019091EE01911116
:1028C00082609091E800977F9093E8008093F100F8
:1028D0001092F100C8C0282F2D7F09F0EAC088238C
:1028E00019F0823061F0E5C08091F301813009F088
:1028F000E0C0933009F080E08093EE012BC080911E
:10290000F301811127C08091F5018F7009F4D1C0C6
:102910008093E9002091EB0020FF1CC0933021F44C
:102920008091EB00806214C09091EB0090619093D5
:10293000EB0021E030E0A90102C0440F551F8A9549
:10294000E2F74093EA001092EA008091EB00886081
:102950008093EB001092E9008091E800877F86C0A9
:102960008111A7C01091F3011F778091E300807857
:10297000812B8093E3008091E800877F8093E800BB
:102980000E943E128091E80080FFFCCF8091E3001E
:1029900080688093E300111102C082E001C083E0EF
:1029A0008093F00186C08058823008F082C0809108
:1029B000F3019091F4018C3D53E0950779F583E0A4
:1029C0008A838AE289834FB7F894DE01139620E068
:1029D0003EE051E2E32FF0E050935700E49120FFF6
:1029E00003C0E295EF703F5FEF708E2F90E0EA300A
:1029F00010F0C79601C0C0968D939D932F5F243130
:102A000049F74FBF8091E800877F8093E8006AE232
:102A100070E0CE0101960E94451114C0AE014F5FD7
:102A20005F4F6091F5010E948C10BC01892B09F465
:102A300040C09091E800977F9093E80089819A8147
:102A40000E94A8118091E8008B778093E80031C044
:102A5000803879F58091E800877F8093E800809145
:102A6000EC018093F1008091E8008E778093E8007C
:102A70000E943E121EC081111CC09091F301923041
:102A8000C0F48091E800877F8093E8009093EC0188
:102A90000E943E128091EC01811106C08091E300FA
:102AA00087FD02C081E001C084E08093F0010E94B4
:102AB000770F8091E80083FF0AC08091E800877F4C
:102AC0008093E8008091EB0080628093EB00AA96EF
:102AD0000FB6F894DEBF0FBECDBFDF91CF911F912F
:102AE0000895CF938091F0018823A1F0C091E9006F
:102AF000CF709091EC00892F817090FD80E8C82BF9
:102B00001092E9008091E80083FD0E942014CF70AC
:102B1000C093E900CF91089590937401809373015D
:102B20000895E0917301F0917401309721F00190C4
:102B3000F081E02D099480E00895EF92FF920F93C9
:102B40001F93CF93DF93E0917301F091740130975D
:102B5000B1F18C010280F381E02D09958091D701BC
:102B600082FF2DC080FF04C08BE896E00E94D4074E
:102B7000E80110E185E8E82E86E0F82E8091D70183
:102B800080FF0BC088811F928F93FF92EF920E946B
:102B90006D080F900F900F900F901150219611110A
:102BA000EDCF8091D70180FF0AC083E896E0DF91E6
:102BB000CF911F910F91FF90EF900C94D407DF916C
:102BC000CF911F910F91FF90EF900895E0917301C5
:102BD000F0917401309721F00480F581E02D099483
:102BE000089520917101309172018217930771F05D
:102BF0009093720180937101E0917301F0917401DF
:102C0000309721F00680F781E02D099408952091F6
:102C10006F01309170018217930771F090937001EA
:102C200080936F01E0917301F0917401309721F06E
:102C30000084F185E02D0994089508950C941D16E3
:102C40000E946F220E94180A0C943523CF93C82F3C
:102C50008091D70182FF1EC080FF04C084EA96E005
:102C60000E94D4078091D70180FF0CC01F92CF93A0
:102C70008FE996E09F938F930E946D080F900F90BD
:102C80000F900F908091D70180FF04C08DE996E0EE
:102C90000E94D4078C2FCF910C94C30DCF92DF925A
:102CA000EF92FF920F931F93CF93DF93CDB7DEB7D1
:102CB0002B970FB6F894DEBF0FBECDBF0E94350A2A
:102CC00086E7C82E81E0D82E00E010E0E02E802FAD
:102CD0000E94610BF60141916F01F42EF826B1F4C8
:102CE0000F5F1F4F0E30110589F78FEF89838A839D
:102CF0001B820E9478228160782F9D838C8349817A
:102D00005A816B818D810E94F11640C09091D7014C
:102D100091FF04C08B870E94670B8B8520E030E019
:102D20004F2D50E0922FBA01022E02C07595679583
:102D30000A94E2F760FF24C02E83EF8221E030E0A6
:102D4000690102C0CC0CDD1C9A95E2F790E08C2161
:102D50009D21892B09F420E028870E947822816038
:102D6000782F9A8789874E815F8168858A850E943E
:102D7000F116F801EA58FE4F8081C826C08206C0CD
:102D80002F5F3F4F2630310569F6AACF0E94A62655
:102D9000109175010E9491151817A1F00E949115CC
:102DA000809375012B960FB6F894DEBF0FBECDBF92
:102DB000DF91CF911F910F91FF90EF90DF90CF9017
:102DC0000C9426162B960FB6F894DEBF0FBECDBF1F
:102DD000DF91CF911F910F91FF90EF90DF90CF90F7
:102DE0000895CF93DF93CDB7DEB72B970FB6F89446
:102DF000DEBF0FBECDBF4F83588769877A878B8729
:102E0000DE01119686E0FD0111928A95E9F785E0D1
:102E1000FE01379601900D928A95E1F749815A811A
:102E20006B817C818D819E810E94071E2B960FB63F
:102E3000F894DEBF0FBECDBFDF91CF910895CF9341
:102E4000882309F4C2C0C82F823859F40E94911512
:102E500081FDBBC089E30E94A3200E94822189E3F7
:102E60000CC0833879F40E94911580FDAEC083E5D3
:102E70000E94A3200E94822183E50E94F620CF9128
:102E80000C948221843859F40E94911582FD9DC0D2
:102E900087E40E94A3200E94822187E4EECF8CEF7A
:102EA0008C0F813A48F48C2F0E94392B81118DC0F0
:102EB0008C2F0E94A320E3CF80E28C0F883048F44F
:102EC000C77081E001C0880FCA95EAF70E944B21C4
:102ED000D6CF8BE58C0F833078F4C53A29F0C63A0B
:102EE00031F083E890E005C081E890E002C082E81C
:102EF00090E0CF910C94F11588E58C0F833108F0A8
:102F000064C0C83A39F1C93A41F1CA3A49F1CB3AF9
:102F100051F1CC3A59F1CD3A61F1C03B69F1CE3A69
:102F200071F1CF3A79F1C13B81F1C23B89F1C33BE9
:102F300091F1C43B99F1C53BA1F1C63BA9F1C73B57
:102F4000B1F1C83BB9F1C93BC1F1CA3BC9F180E05D
:102F500090E038C082EE90E035C089EE90E032C05B
:102F60008AEE90E02FC085EB90E02CC086EB90E0DD
:102F700029C087EB90E026C08CEC90E023C08DEC5C
:102F800090E020C083E891E01DC08AE891E01AC07B
:102F900082E991E017C084E991E014C081E292E0F7
:102FA00011C083E292E00EC084E292E00BC085E2A1
:102FB00092E008C086E292E005C087E292E002C09B
:102FC0008AE292E0CF910C940716CF91089588235E
:102FD00009F44BC0823859F40E94911581FF45C015
:102FE00089E30E94A3200E94822189E30CC08338D8
:102FF00071F40E94911580FF38C083E50E94A320E0
:103000000E94822183E50E94F6200C94822184385C
:1030100059F40E94911582FF28C087E40E94A320E2
:103020000E94822187E4EFCF9CEF980F913A58F3EA
:1030300090E2980F983050F4877091E001C0990F9A
:103040008A95EAF7892F0E945121DFCF9BE5980FDF
:10305000933020F480E090E00C94F115885A83318D
:1030600020F480E090E00C9407160895882321F066
:103070000E944B210C9482210895882321F00E9404
:1030800051210C9482210895BF92CF92DF92EF924A
:10309000FF920F931F93CF93DF9300D000D000D007
:1030A000CDB7DEB725E0FC01DE01119601900D924F
:1030B0002A95E1F7FC014081318102812581229529
:1030C0002F7063817481672B09F4E5C23F3F19F4C7
:1030D0004F3F09F4E0C27C0149833A8389819A8198
:1030E0002E830E946220182FB92E0E9461200E9418
:1030F000281FEB2DE295EF70F0E0E05AFF4F2E8194
:103100000C94372E8B2D807F9B2D9F70F92E88235A
:1031100019F0F29480EFF822002349F0FF2009F41F
:1031200067C28F2D0E945B210E94822161C2812F84
:103130000E94E717FF2009F4AEC28F2D0E94612183
:1031400026960FB6F894DEBF0FBECDBFDF91CF91AC
:103150001F910F91FF90EF90DF90CF90BF900C9454
:1031600082213B2D307F8B2D8F70303211F0829574
:10317000807F112319F0113021F12CC00023B9F008
:10318000222309F4A0C1213009F09DC126960FB673
:10319000F894DEBF0FBECDBFDF91CF911F910F918D
:1031A000FF90EF90DF90CF90BF900C946B21222383
:1031B00019F0213009F46FC28E830E946E218E8136
:1031C00096C1002321F0223008F065C27CC1211194
:1031D00062C28DC1002321F0222309F474C108C208
:1031E000222309F484C119C22B2D2695269523701C
:1031F00030E02115310521F021303105D1F04BC2ED
:10320000002321F0812F9B2D937002C080E090E07D
:1032100026960FB6F894DEBF0FBECDBFDF91CF91DB
:103220001F910F91FF90EF90DF90CF90BF900C9483
:10323000F115002321F0812F9B2D937002C080E0B7
:1032400090E026960FB6F894DEBF0FBECDBFDF919B
:10325000CF911F910F91FF90EF90DF90CF90BF9093
:103260000C940716812F002319F00E942C2502C010
:103270000E94942526960FB6F894DEBF0FBECDBFF0
:10328000DF91CF911F910F91FF90EF90DF90CF9042
:10329000BF900C9419268B2D837009F07BC001110F
:1032A000FAC1812F829586958770880F880F912F9C
:1032B0009F70C92ED12CE12CF12C082E04C0CC0C0F
:1032C000DD1CEE1CFF1C0A94D2F714FF12C04FE065
:1032D00050E060E070E004C0440F551F661F771F88
:1032E0008A95D2F7CB01BA0160957095809590953B
:1032F00003C060E070E0CB012B2D2695269523704E
:10330000422F50E042305105D9F04330510569F168
:103310006C297D298E299F294130510551F126962E
:103320000FB6F894DEBF0FBECDBFDF91CF911F91D6
:103330000F91FF90EF90DF90CF90BF900C944F1FB4
:103340006C297D298E299F2926960FB6F894DEBF19
:103350000FBECDBFDF91CF911F910F91FF90EF90E6
:10336000DF90CF90BF900C946B1F0E944F1FC7013E
:10337000B60126960FB6F894DEBF0FBECDBFDF9123
:10338000CF911F910F91FF90EF90DF90CF90BF9062
:103390000C94331F002319F08B2D817001C086958A
:1033A000882309F478C1812F829586958770880FCC
:1033B000880F912F9F70C92ED12CE12CF12C082E53
:1033C00004C0CC0CDD1CEE1CFF1C0A94D2F714FFC9
:1033D00012C04FE050E060E070E004C0440F551FA1
:1033E000661F771F8A95D2F7CB01BA016095709559
:1033F0008095909503C060E070E0CB012B2D269561
:1034000026952370422F50E042305105D9F04330C9
:10341000510569F16C297D298E299F29413051057B
:1034200051F126960FB6F894DEBF0FBECDBFDF91E7
:10343000CF911F910F91FF90EF90DF90CF90BF90B1
:103440000C9429206C297D298E299F2926960FB658
:10345000F894DEBF0FBECDBFDF91CF911F910F91CA
:10346000FF90EF90DF90CF90BF900C9445200E948A
:103470002920C701B60126960FB6F894DEBF0FBE0D
:10348000CDBFDF91CF911F910F91FF90EF90DF9013
:10349000CF90BF900C940D20103FD1F118F4103E46
:1034A00050F4A1C0123F09F463C008F44CC0133FAC
:1034B00009F473C098C01F708B2D8F710023A1F089
:1034C0000E94A61F812F26960FB6F894DEBF0FBE6E
:1034D000CDBFDF91CF911F910F91FF90EF90DF90C3
:1034E000CF90BF900C9436180E94C71F812F26964C
:1034F0000FB6F894DEBF0FBECDBFDF91CF911F9105
:103500000F91FF90EF90DF90CF90BF900C943D18FB
:103510000023A9F02111BFC08B2D8F7126960FB605
:10352000F894DEBF0FBECDBFDF91CF911F910F91F9
:10353000FF90EF90DF90CF90BF900C94EC1F223063
:1035400008F0A9C0E9CF0023A9F08B2D8F71269632
:103550000FB6F894DEBF0FBECDBFDF91CF911F91A4
:103560000F91FF90EF90DF90CF90BF900C94A61F2B
:10357000002359F38B2D8F7126960FB6F894DEBF7A
:103580000FBECDBFDF91CF911F910F91FF90EF90B4
:10359000DF90CF90BF900C94C71F002399F08B2D24
:1035A0008F7126960FB6F894DEBF0FBECDBFDF91A8
:1035B000CF911F910F91FF90EF90DF90CF90BF9030
:1035C0000C94911F26960FB6F894DEBF0FBECDBFA8
:1035D000DF91CF911F910F91FF90EF90DF90CF90EF
:1035E000BF900C94871F0023A9F0222309F4ADCFCC
:1035F000812F26960FB6F894DEBF0FBECDBFDF91A8
:10360000CF911F910F91FF90EF90DF90CF90BF90DF
:103610000C941F17222309F4ADCF812F26960FB6E5
:10362000F894DEBF0FBECDBFDF91CF911F910F91F8
:10363000FF90EF90DF90CF90BF900C94E7174B2D49
:103640004F70612FC7010E94760826960FB6F89436
:10365000DEBF0FBECDBFDF91CF911F910F91FF90C5
:10366000EF90DF90CF90BF900C94AB1E4B2D4F701E
:10367000612FC70126960FB6F894DEBF0FBECDBFEF
:10368000DF91CF911F910F91FF90EF90DF90CF903E
:10369000BF900C946D0C26960FB6F894DEBF0FBE4B
:1036A000CDBFDF91CF911F910F91FF90EF90DF90F1
:1036B000CF90BF9008950E9468210E943D210E94F2
:1036C00082210E944C270E94192680E090E00E94EF
:1036D000F11580E090E00C9407160E9458210C949C
:1036E0005B1B0E946220292F22952F7030E02C3026
:1036F00031054CF42A3031056CF422503109223066
:10370000310588F407C02C30310549F02F303105E0
:1037100031F009C0803E48F0803F29F406C093FB99
:10372000882780F9089580E0089581E00895CF9377
:10373000DF9300D000D01F92CDB7DEB70F900F906F
:103740000F900F900F90DF91CF910895CF93DF935B
:1037500000D000D000D0CDB7DEB726960FB6F894D3
:10376000DEBF0FBECDBFDF91CF9108951F93CF93E2
:10377000DF93C091840116E080918501C81799F00C
:10378000D0E01C9FF0011D9FF00D1124EA57FE4F61
:103790004081518162817381848195810E94A61B41
:1037A0002196C770E9CFDF91CF911F910895409185
:1037B000B6015091B7016091B8017091B901809143
:1037C000BA019091BB010C94A61B8091BB0182951C
:1037D0008F7009F054C08091B801882309F44FC05C
:1037E00080918401A09185016091B6017091B7012B
:1037F0004091B9015091BA01B6E08A1709F43FC06F
:1038000090E041155105C1F17F3F11F46F3FA1F1E7
:10381000B89FF001B99FF00D1124EA57FE4F2181A6
:1038200072132AC02081621327C02281211124C073
:10383000238134812417350710F421503109241BCA
:10384000350B283C3105C0F42091BB012F7020615D
:103850002093BB0126E0289FF001299FF00D112441
:10386000E557FE4F80818F708061808386EB91E009
:103870000E9444180C94B61B01968770BECF089521
:10388000CF92DF92EF92FF920F931F93CF93DF932C
:10389000CDB7DEB762970FB6F894DEBF0FBECDBFCF
:1038A0008C0185E0F801DE011D9601900D928A954C
:1038B000E1F7D8014C9111965C91119712966C9199
:1038C00012971396CD90DC9014973091B6017091B9
:1038D000B7018091B9019091BA01009709F46BC1C9
:1038E0007F3F19F43F3F09F466C1E090B801EE2034
:1038F00009F4C0C02091BB01C816D90628F0F60112
:10390000E81BF90BCF0104C0809590958C0D9D1D8F
:10391000FF24F394883C910578F0F12C207F09F086
:10392000C6C07C2DD98AC88A89890E94971B86EBDC
:1039300091E00E944418B1C0822F807F09F046C0F8
:10394000751314C0341312C0611110C02F702061A0
:103950002093BB010E94D71B86EB91E00E94441884
:103960008091BB01D80115968C932EC0CD2819F1FA
:103970005F3F11F44F3FF9F0F62E61111CC08091AA
:1039800084012091850136E0821709F45AC090E045
:10399000389FF001399FF00D1124EA57FE4F7181D5
:1039A000571306C07081471303C07281711103C0A1
:1039B00001968770E9CFF62E662309F418C180912D
:1039C000BB0181608093BB01F12C11C1751308C04C
:1039D000341306C0611104C08091BB01D801C3C07B
:1039E0004D875E878D859E856A8B0E94711B6A89D3
:1039F0008823E1F16623D1F12091BB01822F8295CA
:103A00008F7090E0029774F08091B6019091B701A9
:103A100098878F831986DB86CA862C87CE01079606
:103A20000E94441886E0F801A6EBB1E001900D92E7
:103A30008A95E1F70E94E51B0E94D71BFF24F394AF
:103A4000D6C04D875E878D859E850E946220292F76
:103A500022952F7030E0223031050CF0BCC09F70F1
:103A600009F0B6C0805E883008F4C1C0C8010E9469
:103A70004418E4CFC816D90608F453C0F601E81B71
:103A8000F90BCF01883C910508F450C0F12C7C2D36
:103A9000D98AC88A89890E94971BE6EBF1E086E003
:103AA000DF011D928A95E9F70E94D71BA0C075130C
:103AB00014C0341312C0611110C08091BB01F80111
:103AC0008583C8010E94441886E0E6EBF1E0DF013F
:103AD0001D928A95E9F7FE2C8AC04D875E878D85F9
:103AE0009E856A8B0E94711B6A89882309F4BECF68
:103AF000662309F4BBCF2091BB01822F82958F7082
:103B000090E002970CF48ECF8091B6019091B701AE
:103B10009A8389831B82DD82CC822E83CE0101961B
:103B20007FCF809590958C0D9D1DACCFF62E662392
:103B300009F49CCF75132EC034132CC02091BB0107
:103B400020FD1FC0822F82958F70D9F0D801159665
:103B50002C9315978F3049F08F5F982F9295907F17
:103B6000822F8F70892B15968C93C8010E94441860
:103B700086E0F801A6EBB1E001900D928A95E1F79D
:103B800093CF86E0F801A6EBB1E001900D928A9503
:103B9000E1F72DC04D875E878D859E850E94711B44
:103BA000811140CF8091BB0181608093BB01C8012E
:103BB0000E9444181CC0662309F458CF4D875E87C5
:103BC0008D859E850E94711B882309F44FCF2ACFD3
:103BD000811148CF0CC0243031050CF047CF9F70C5
:103BE00009F440CFF8019581907F09F03BCF8F2DEC
:103BF00062960FB6F894DEBF0FBECDBFDF91CF91B6
:103C00001F910F91FF90EF90DF90CF9008951F9339
:103C1000CF93DF93CDB7DEB72C970FB6F894DEBF06
:103C20000FBECDBF4F83588769877A878B879C8764
:103C3000CE0107960E94401C882369F08F819885E9
:103C40002A853B85232BF1F19F3F09F063C08F3F0D
:103C500009F060C037C086E0FE013796DE0111969C
:103C600001900D928A95E1F76F817885EA85FB8551
:103C7000309741F17F3F11F46F3F21F12091850191
:103C800030E0C9010196877099274091840150E086
:103C90008417950709F447C069837A83FD83EC8311
:103CA00096E0929FD001939FB00D1124AA57BE4F6A
:103CB000FE01319601900D929A95E1F7809385016E
:103CC0000E94B61B16E080918401909185018917AE
:103CD000C1F1189FC00111248A579E4F0E94401CB9
:103CE000882379F1E09184011E9FF0011124EA57A5
:103CF000FE4F4081518162817381848195810E9450
:103D0000A61B8091840190E001968770992780938B
:103D10008401D9CF4F81588569857A858B859C85AB
:103D20000E94A61BCFCF0E946D1B1092850110929E
:103D30008401E6EBF1E086E0DF011D928A95E9F768
:103D4000C1CF2C960FB6F894DEBF0FBECDBFDF916A
:103D5000CF911F910895EF92FF920F931F93CF93EE
:103D6000DF938C01892B09F46CC0F12CEE24E394D1
:103D7000E8012196F8018491843740F4843008F0FA
:103D800051C0813081F0823019F15BC0853709F470
:103D900044C0A8F19CE7980F903708F052C08F7785
:103DA0000E94E71741C00E5F1F4FFE01C49180E2E1
:103DB0008C0F883048F4C7708E2D01C0880FCA95CB
:103DC000EAF70E945B2114C08C2F0E941F172DC0A0
:103DD0000E5F1F4FFE01C49180E28C0F883058F4B3
:103DE000C7708E2D01C0880FCA95EAF70E94612125
:103DF0000E9482211AC08C2F0E94E71716C00E5F06
:103E00001F4FFE01C491CC2381F08FE99FE0019701
:103E1000F1F700C00000C150F6CF0E5F1F4FFE014A
:103E2000F49003C00E941F178E018F2D882309F480
:103E30009FCFEFE9FFE03197F1F700C0000081501C
:103E4000F5CFDF91CF911F910F91FF90EF900895E3
:103E500008956093C0017093C1018093C201909353
:103E6000C3010C945B1B0F931F930091C001109131
:103E7000C1012091C2013091C301DC01CB01802B33
:103E8000912BA22BB32B8093C0019093C101A093DF
:103E9000C201B093C3011F910F910C945B1B0F9350
:103EA0001F930091C0011091C1012091C201309176
:103EB000C301DC01CB0180239123A223B323809390
:103EC000C0019093C101A093C201B093C3011F919F
:103ED0000F910C945B1B0F931F930091C0011091E5
:103EE000C1012091C2013091C301DC01CB018027C7
:103EF0009127A227B3278093C0019093C101A0937B
:103F0000C201B093C3011F910F910C945B1B1092DF
:103F1000BC011092BD011092BE011092BF010C9421
:103F20005B1B41E050E060E070E004C0440F551FAF
:103F3000661F771F8A95D2F74093BC015093BD014D
:103F40006093BE017093BF010C945B1B41E050E095
:103F500060E070E004C0440F551F661F771F8A950C
:103F6000D2F78091BC019091BD01A091BE01B091AA
:103F7000BF01482B592B6A2B7B2B4093BC015093DC
:103F8000BD016093BE017093BF010C945B1B41E0C7
:103F900050E060E070E004C0440F551F661F771FBB
:103FA0008A95D2F740955095609570958091BC01A7
:103FB0009091BD01A091BE01B091BF01482359234A
:103FC0006A237B234093BC015093BD016093BE01E3
:103FD0007093BF010C945B1B41E050E060E070E027
:103FE00004C0440F551F661F771F8A95D2F7809132
:103FF000BC019091BD01A091BE01B091BF014827C5
:1040000059276A277B274093BC015093BD016093D9
:10401000BE017093BF010C945B1B0F931F93009123
:10402000BC011091BD012091BE013091BF01DC01A6
:10403000CB01802B912BA22BB32B8093BC019093AF
:10404000BD01A093BE01B093BF011F910F910C94CD
:104050005B1B0F931F930091BC011091BD01209138
:10406000BE013091BF01DC01CB0180239123A2234B
:10407000B3238093BC019093BD01A093BE01B09384
:10408000BF011F910F910C945B1B0F931F93009125
:10409000BC011091BD012091BE013091BF01DC0136
:1040A000CB0180279127A227B3278093BC0190934F
:1040B000BD01A093BE01B093BF011F910F910C945D
:1040C0005B1B0895CF92DF92EF92FF920F931F93A5
:1040D000CF93DF938C01C090C001D090C101E090DC
:1040E000C201F090C3014091BC015091BD016091AB
:1040F000BE017091BF01C42AD52AE62AF72ACFE172
:10410000D0E0D701C6010C2E04C0B695A7959795AF
:1041100087950A94D2F780FF07C0B8018C2F0E94C0
:10412000900C8130910531F4219758F7B80180E067
:104130000E94900CDF91CF911F910F91FF90EF9013
:10414000DF90CF90089590910C01992321F09091E8
:104150000D01911109C020910E0130910F01F9015B
:1041600032969FEF40E030C0982F969596959695A1
:104170009F30A0F4E0910E01F0910F01E90FF11DC5
:10418000877021E030E0A90102C0440F551F8A95D5
:10419000E2F7CA019181892B818308959091D7011B
:1041A00090FF23C01F928F9385ED96E09F938F938E
:1041B0000E946D080F900F900F900F9008959F3FF1
:1041C00039F04F5F4E3041F051915813F8CF0DC088
:1041D0005111F7CF942FF5CF9F3F39F0F901E90F37
:1041E000F11D97FDFA9582830895089590910C0131
:1041F000992321F090910D01911109C020910E0198
:1042000030910F01F9013296205F3F4F30C0982F57
:104210009695969596959F30A8F4E0910E01F091B1
:104220000F01E90FF11D877021E030E0A90102C004
:10423000440F551F8A95E2F7CA0180959181892321
:10424000818308959091D70190FF16C01F928F939C
:1042500087EB96E09F938F930E946D080F900F90CD
:104260000F900F9008953196E217F30729F090818F
:104270009813F9CF1082F7CF089581E090E0E09194
:104280000E01F0910F01E80FF91F108201968031A5
:104290009105A9F708959091D601892B8093D601B5
:1042A000089580959091D60189238093D601089531
:1042B0001092D60108959091D501892B8093D50154
:1042C000089580959091D50189238093D501089513
:1042D0001092D50108958093C40108951092C401ED
:1042E000089580910E0190910F01FC0131969C017F
:1042F000205F3F4F80E0919191118F5FE217F307AC
:10430000D1F70895E0910E01F0910F018091D6014F
:104310008083E0910E01F0910F0190818091D50191
:10432000892B80838091C401882361F0E0910E0184
:10433000F0910F019081892B80830E94712181115E
:104340001092C40180910E0190910F010C949D1563
:1043500090933B0180933A010895CF92DF92EF92C0
:10436000FF926C01EE24FF24C114D104E104F10496
:1043700021F0C701B60120E101C020E0C72ED82EF0
:10438000E92EFF24C114D104E104F10419F0285FDF
:10439000C701B6016B017C0154E0F694E794D79411
:1043A000C7945A95D1F7C114D104E104F10419F06E
:1043B0002C5FC701B6016B017C0142E0F694E794E3
:1043C000D794C7944A95D1F7C114D104E104F104FC
:1043D00019F02E5FC701B601DC01CB01B695A79598
:1043E00097958795892B8A2B8B2B09F02F5F822F2E
:1043F000FF90EF90DF90CF9008958295982F9C7C4E
:10440000392F36953695282F237344E0249FC00119
:104410001124932F982B292F2A7A2695892F857579
:10442000880F822B08951F93CF93DF931F92CDB7F0
:10443000DEB799830E94FD21182F9981892F0E9450
:10444000FD21212F30E0322F2227A901482BCA015C
:104450000F90DF91CF911F9108958091F0018430EA
:1044600009F11092D80120E488E190E00FB6F894A9
:10447000A895809360000FBE2093600083B7817F72
:10448000846083BF83B7816083BF7894889583B746
:104490008E7F83BF88E10FB6F894809360001092FE
:1044A00060000FBE089508950895CF930E9453228F
:1044B0000E94350A0E945422C0E08C2F0E94610B9A
:1044C000811104C0CF5FCE30C1F701C081E0CF9130
:1044D00008950E946D1B0E9491150C94C30D82E0FB
:1044E00084BD93E095BD9AEF97BD80936E000895CB
:1044F0002FB7F8948091D9019091DA01A091DB0156
:10450000B091DC012FBF0895CF92DF92EF92FF921E
:104510000F931F932FB7F8944091D9015091DA016E
:104520006091DB017091DC012FBF6A017B01EE24F9
:10453000FF248C0120E030E0C016D106E206F3062D
:1045400010F4415051099A01281B390BC9011F91E0
:104550000F91FF90EF90DF90CF9008951F920F92F0
:104560000FB60F9211248F939F93AF93BF938091B7
:10457000D9019091DA01A091DB01B091DC010196A3
:10458000A11DB11D8093D9019093DA01A093DB01A5
:10459000B093DC01BF91AF919F918F910F900FBEAF
:1045A0000F901F9018950E948F12F8942FEF87EAB2
:1045B00091E6215080409040E1F700C0000087E084
:1045C00090EBDC018093F9019093FA01A093FB0139
:1045D000B093FC019CE088E10FB6F894A895809315
:1045E00060000FBE90936000FFCFEF92FF920F9399
:1045F0001F93CF93DF93D82FC0E08C2F0E94610BC5
:1046000000E010E0E82EF12CC701002E02C09595C5
:1046100087950A94E2F780FD06C00F5F1F4F0630B2
:10462000110591F709C0602F7C2F80E00E946E0C6D
:10463000D813F3CF81E004C0CF5FCE30F1F680E035
:10464000DF91CF911F910F91FF90EF900895CF933D
:10465000C82F8CE20E94F522882321F08C2FCF9165
:104660000C94F52280E0CF910895CF930E9484248A
:10467000811102C00E946A248AEF96E00E94D4074A
:10468000C5E6C15049F00E94350A8FE39CE90197C5
:10469000F1F700C00000F5CF83EF96E00E94D40749
:1046A00089E20E942723811113C18AE20E942723F5
:1046B00081110E946A2485E00E94272381110E94B3
:1046C000D3220E948F248093D70187E00E94272362
:1046D0008823A9F18BE10E942723882351F0809140
:1046E000D70181FB222720F991E0922790FB81F9E5
:1046F0000EC08EE00E942723882361F08091D701AD
:1047000082FB222720F991E0922790FB82F9809387
:10471000D70115C080E10E9427239091D7018823FB
:1047200041F093FB222720F981E0822780FB93F957
:1047300004C0892F809580FB90F99093D7018091D8
:10474000D7010E9493240E94A1248093EA0180EE65
:104750000E942723882341F08091EA01982F9095A9
:1047600090FB80F98093EA0189E30E942723882344
:1047700059F08091EA0181FB222720F991E09227EC
:1047800090FB81F98093EA0182EE0E94272388231F
:1047900059F08091EA0182FB222720F991E09227CB
:1047A00090FB82F98093EA0186EE0E9427238823FA
:1047B00059F08091EA0183FB222720F991E09227AA
:1047C00090FB83F98093EA0183EE0E9427238823DC
:1047D00059F08091EA0184FB222720F991E0922789
:1047E00090FB84F98093EA0185E30E9427238823C4
:1047F00059F08091EA0185FB222720F991E0922768
:1048000090FB85F98093EA0181E30E9427238823A6
:1048100059F08091EA0186FB222720F991E0922746
:1048200090FB86F98093EA0181E10E942723882387
:1048300059F08091EA0187FB222720F991E0922725
:1048400090FB87F98093EA018091EA010E94A524F8
:104850008091EA0187FB882780F980930D0187E228
:104860000E942723C82F8EE10E9427238111C26056
:104870008FE10E9427238111C46080E20E942723D8
:104880008111C86081E20E9427238111C06182E208
:104890000E9427238111C06283E20E942723811195
:1048A000C06484E20E942723882311F0C06802C0FC
:1048B000CC2329F08C2F0E949C246C2F03C00E94D3
:1048C0009824682F70E080E090E0CF910C94291F2D
:1048D000CF9108956DEE7EEF80E090E00E946D2E06
:1048E00060E082E090E00E945F2E60E083E090E074
:1048F0000E945F2E60E084E090E00E945F2E60E006
:1049000085E090E00C945F2E80E090E00E94592EAC
:1049100021E08D3E9E4F09F020E0822F089582E035
:1049200090E00C94512E682F82E090E00C945F2E62
:1049300083E090E00C94512E682F83E090E00C947B
:104940005F2E84E090E00C94512E682F84E090E07C
:104950000C945F2E8091DF0180FF0BC060911301EA
:1049600085E0689FB00111247595679575956795E9
:104970002BC081FF09C06091130185E0689FB001E1
:1049800011247595679520C082FF07C060911301BF
:1049900085E0689FB001112417C09091E001992330
:1049A000D1F060911201961788F72091130185E0EC
:1049B000289F90011124929FA001939F500D1124D4
:1049C00070E0CA010E94232E6038710540F4611521
:1049D000710539F002C065E070E0862F08958FE719
:1049E000089581E008958091DF0180FF08C0609103
:1049F000110170E0759567957595679521C081FFE8
:104A000006C06091110170E07595679519C082FF2D
:104A100004C06091110170E010C09091E0019923F1
:104A2000C1F0609110019617A0F780911101899F44
:104A3000C001112470E00E94232E6038710528F413
:104A40006115710521F0862F08958FE7089581E0A3
:104A5000089561E070E0F4CF803F21F40E94AA2421
:104A6000819504C0813F29F40E94AA248093E30128
:104A70000895823F21F40E94AA24819504C0833FB7
:104A800029F40E94AA248093E2010895893F19F431
:104A90000E94F32405C08A3F31F40E94F3248195DB
:104AA0008093E40108958B3F21F40E94F3248195C3
:104AB00004C08C3F29F40E94F3248093E5010895FB
:104AC000843F21F48091E101816017C0853F21F48A
:104AD0008091E101826011C0863F21F48091E10163
:104AE00084600BC0873F21F48091E101886005C09C
:104AF000883F31F48091E10180618093E101089564
:104B00008D3F21F48091DF0181600BC08E3F21F445
:104B10008091DF01826005C08F3F29F48091DF0121
:104B200084608093DF010895803F39F48091E30130
:104B300087FF6CC01092E30169C0813F29F4809126
:104B4000E3011816BCF362C09091E201823F29F4A0
:104B500097FF5CC01092E20159C0833F19F4191607
:104B6000CCF354C0893F41F48091E40118160CF055
:104B70004DC01092E4014AC08A3F29F48091E401BB
:104B800087FF44C0F6CF8B3F39F48091E50187FF62
:104B90003DC01092E5013AC08C3F29F48091E501B7
:104BA0001816BCF333C0843F21F48091E1018E7F5D
:104BB00017C0853F21F48091E1018D7F11C0863FB0
:104BC00021F48091E1018B7F0BC0873F21F480911C
:104BD000E101877F05C0883F31F48091E1018F7E3C
:104BE0008093E10113C08D3F21F48091DF018E7F1E
:104BF0000BC08E3F21F48091DF018D7F05C08F3F78
:104C000029F48091DF018B7F8093DF018091E201A5
:104C100081110EC08091E30181110AC08091E401ED
:104C2000811106C08091E501811102C01092E0015E
:104C300008958091D70183FF7EC086E397E00E94AC
:104C4000D4078091E1011F928F9381E397E09F93B6
:104C50008F930E946D088FE297E00E94D4078091A5
:104C6000E201282F332727FD30953F938F938CE265
:104C700097E09F938F930E946D088AE297E00E94CD
:104C8000D4078091E301282F332727FD30953F93E8
:104C90008F9387E297E09F938F930E946D0885E240
:104CA00097E00E94D4078091E401282F332727FD45
:104CB00030953F938F9382E297E09F938F930E946A
:104CC0006D0880E297E00E94D4078091E501282FCB
:104CD000332727FD30953F938F938DE197E09F9386
:104CE0008F930E946D088AE197E00E94D40780911B
:104CF000E0011F928F9387E197E09F938F930E942B
:104D00006D0885E197E00E94D4078091DF011F9232
:104D10008F9382E197E09F938F930E946D088FE0BD
:104D200097E00E94D4078DB79EB74C960FB6F894C3
:104D30009EBF0FBE8DBF81EE91E00E94E6150E94DE
:104D400078229093DE018093DD0108951F93CF9325
:104D5000DF938091DD019091DE010E948422AC01FD
:104D60009091E001992321F02091140130E006C0D8
:104D7000209115018AE0289F9001112442175307C2
:104D800008F486C08091E201C091E301D091E40172
:104D90001091E501811107C0C11176C0D11174C015
:104DA000111172C075C09F3F19F09F5F9093E00191
:104DB000181624F40E94AA248093E2018091E20153
:104DC00087FF05C00E94AA2481958093E2011C16EA
:104DD00024F40E94AA248093E3018091E30187FFD9
:104DE00005C00E94AA2481958093E3016091E201AD
:104DF000662339F1C091E301CC2319F1772767FDD0
:104E00007095872F972F0E94282D23E333E343E3E8
:104E10005FE30E948C2D0E94F52C6093E2016C2FC1
:104E2000772767FD7095872F972F0E94282D23E302
:104E300033E343E35FE30E948C2D0E94F52C6093E3
:104E4000E3011D1624F40E94F3248093E401809171
:104E5000E40187FF05C00E94F32481958093E4015B
:104E6000111624F40E94F3248093E5018091E5015A
:104E700087FF05C00E94F32481958093E501DF91AF
:104E8000CF911F910C9419269F3F09F08ECF96CF9A
:104E9000DF91CF911F910895E1EEF1E085E0DF0110
:104EA0001D928A95E9F71092E0011092DF010895B2
:104EB00089E599E00E94D4071F9281E08F931F92A9
:104EC00085E08F938BE099E09F938F930E946D080C
:104ED0000F900F900F900F900F900F9008958330C8
:104EE000E9F128F4813061F0823009F108958530CC
:104EF00009F462C008F449C0863009F474C008950A
:104F000080911501262F30E0280F311D2F3F3105EC
:104F100024F4680F6093150103C08FEF809315018F
:104F2000809115011F928F9384E498E072C0809164
:104F30001401262F30E0280F311D2F3F310524F4B6
:104F4000680F6093140103C08FEF80931401809168
:104F500014011F928F9382E398E05BC0809113014C
:104F6000262F30E0280F311D2F3F310524F4680F24
:104F70006093130103C08FEF80931301809113019D
:104F80001F928F938FE198E044C080911201262FE9
:104F900030E0280F311D2F3F310524F4680F609356
:104FA000120103C08FEF80931201809112011F92B2
:104FB0008F938AE098E02DC080911101262F30E078
:104FC000280F311D2F3F310524F4680F6093110124
:104FD00003C08FEF80931101809111011F928F9375
:104FE00081EF97E016C080911001262F30E0280F46
:104FF000311D2F3F310524F4680F6093100103C069
:105000008FEF80931001809110011F928F9386ED96
:1050100097E09F938F930E946D080F900F900F90D1
:105020000F900895833081F128F4813059F0823057
:10503000D1F00895853009F449C0B8F1863009F4FB
:1050400056C0089580911501681720F4861B80933F
:10505000150102C010921501809115011F928F93C6
:1050600087EC97E054C080911401681720F4861BE8
:105070008093140102C010921401809114011F92B8
:105080008F9385EB97E043C080911301681720F45C
:10509000861B8093130102C01092130180911301AB
:1050A0001F928F9382EA97E032C0809112016817B5
:1050B00020F4861B8093120102C01092120180918D
:1050C00012011F928F938DE897E021C0809111010A
:1050D000681720F4861B8093110102C01092110101
:1050E000809111011F928F9384E797E010C0809107
:1050F0001001681720F4861B8093100102C01092E3
:105100001001809110011F928F9389E597E09F9382
:105110008F930E946D080F900F900F900F9008953D
:10512000CF93C82F1F928F938EE59AE09F938F9312
:105130000E946D0881E090E0A0E0B0E0BC01CD01EC
:1051400004C0660F771F881F991FCA95D2F70E9467
:10515000291F0F900F900F900F90CF910C946D1B03
:10516000CF938D3109F465C0B0F58E3009F4CCC110
:1051700000F5873009F49BC1A8F4863009F06DC2B0
:105180008091D701817F8E7F8093D70183E69AE05B
:105190000E94D40785EA9EE00E94D40781E08093B4
:1051A000E70180C1883009F44FC08B3009F47CC11D
:1051B00054C2863109F4F0C138F4803109F4B8C121
:1051C000813109F430C249C2893109F4CEC18B3131
:1051D00009F486C142C2853309F437C248F48732E4
:1051E00009F433C208F433C2893209F42EC235C23D
:1051F000833438F48A3308F02CC2883309F454C15C
:105200002CC2833409F421C2883409F026C20E94DA
:105210006D1B84E99EE00E94D4079FEF23ED80E39D
:10522000915020408040E1F700C000000E94D3224E
:1052300039C184EB9EE00E94D4070E94AF2C0E94EB
:1052400091150E94C30D2EC189EA9EE00E94D407E9
:1052500084E79CE00E94D4070E9498241F928F93B9
:1052600081E79CE09F938F930E946D088FE69CE0FE
:105270000E94D4070E948F24C82F8CE59CE00E94D6
:10528000D4071F92CF9387E59CE09F938F930E9452
:105290006D0885E59CE00E94D4078BE49CE00E94A9
:1052A000D4078C2F81701F928F9388E49CE09F938A
:1052B0008F930E946D0886E49CE00E94D4078CE3E3
:1052C0009CE00E94D407C1FB882780F91F928F932E
:1052D00089E39CE09F938F930E946D0887E39CE095
:1052E0000E94D4078BE29CE00E94D407C2FB88276F
:1052F00080F91F928F9388E29CE09F938F930E9486
:105300006D0886E29CE00E94D4078DE19CE00E943B
:10531000D407C3FBCC27C0F91F92CF938AE19CE04E
:105320009F938F930E946D0888E19CE00E94D407B0
:105330000E94A124C82F84E09CE00E94D4071F9201
:10534000CF938FEF9BE09F938F930E946D088DEF1B
:105350009BE00E94D40784EE9BE00E94D4078C2F30
:1053600081701F928F9381EE9BE09F938F930E9499
:105370006D088DB79EB780960FB6F8949EBF0FBE8E
:105380008DBF8FED9BE00E94D40788EC9BE00E94CC
:10539000D407C1FB882780F91F928F9385EC9BE08F
:1053A0009F938F930E946D0883EC9BE00E94D4072B
:1053B00081EB9BE00E94D407C2FB882780F91F92F3
:1053C0008F938EEA9BE09F938F930E946D088CEAE7
:1053D0009BE00E94D4078AE99BE00E94D407C3FBAC
:1053E000882780F91F928F9387E99BE09F938F9383
:1053F0000E946D0885E99BE00E94D4078BE89BE042
:105400000E94D407C4FB882780F91F928F9388E8F5
:105410009BE09F938F930E946D0886E89BE00E941B
:10542000D40784E79BE00E94D407C5FB882780F956
:105430001F928F9381E79BE09F938F930E946D084B
:105440008FE69BE00E94D40783E59BE00E94D4078F
:10545000C6FB882780F91F928F9380E59BE09F937E
:105460008F930E946D088EE49BE00E94D40786E42F
:105470009BE00E94D407C7FBCC27C0F91F92CF93B3
:1054800083E49BE09F938F930E946D0881E49BE0EF
:105490000E94D4078DB79EB74C960FB6F8949EBF66
:1054A0000FBE8DBFC1E0DEC08AE89AE05BC080918C
:1054B000D701C82FC17080FF09C087E89EE00E9415
:1054C000D4078091D701817F8E7F47C08BE79EE014
:1054D0000E94D4078091D70181608093D701E2CFE9
:1054E0009091D70191FBCC27C0F981E0C827892F83
:1054F000C0FB81F98093D701CC2319F08EE69EE0A2
:1055000027C080E69EE02EC09091D70192FBCC2769
:10551000C0F981E0C827892FC0FB82F98093D701A9
:10552000CC2319F081E59EE013C081E49EE01AC00F
:105530009091D70193FBCC27C0F981E0C827892F30
:10554000C0FB83F98093D701CC2351F085E39EE023
:105550000E94D4078091D70181608093D70182C0D7
:1055600088E29EE00E94D4079DCF89E19EE00E94E0
:10557000D4078DEE9DE00E94D40780EB9DE00E9451
:10558000D40783E89DE00E94D4078FE39DE00E944A
:10559000D40784E19DE0E6CF86E09DE00E94D40739
:1055A0000E9491151F928F938CEE9CE09F938F9396
:1055B0000E946D0880910C011F928F9385ED9CE0F5
:1055C0009F938F930E946D0880916E011F928F931D
:1055D00082EC9CE09F938F930E946D0880910D0157
:1055E0001F928F938FEA9CE09F938F930E946D0888
:1055F0008091D9019091DA01A091DB01B091DC0199
:10560000BF93AF939F938F938BE99CE09F938F936E
:105610000E946D088DB79EB746960FB6F8949EBF50
:105620000FBE8DBF3FCF0E946D1BC0910D0181E069
:10563000C827C0930D01CC2329F081E99CE00E948A
:10564000D40710C086E89CE08DCF80E003C08D5168
:1056500001C089530E94902825CF84E89CE00E94D5
:10566000D407C0E08C2FCF91089580E0089580E0AA
:105670000895CF93C82F8091E701813081F020F009
:10568000823009F44FC045C1E0910E01F0910F0145
:105690008081813169F0823209F03DC109C0E09119
:1056A0000E01F0910F018081813111F0823261F49D
:1056B0008C2F0E94352B811104C08C2F0E94B028A2
:1056C0002FC081E090E02CC08C2F0E94372B8111DD
:1056D00026C0C431E1F070F4CB3081F0C031D1F498
:1056E0000E94582786E59AE00E94D40782E08093C2
:1056F000E70115C0C93259F0C83361F483E69AE076
:105700000E94D4078AE59AE00E94D40708C010924C
:10571000E70103C184E59AE00E94D407FEC081E05E
:105720008170FDC0C43220F5CE3108F0C0C0CB304E
:1057300099F1C8F4C73009F0D2C08AE0809315010E
:1057400094E19093140193E09093130180931201DC
:1057500088E08093110188E2809310018AEF98E03D
:105760000E94D407BFC0C33149F1C431C1F0B7C0F2
:10577000CB3409F4A9C028F4C93289F0C83361F0E8
:10578000AEC0C13509F49EC0C23509F499C0CE340B
:1057900009F0A5C06AE09EC00E945827A3C080916E
:1057A000E601882319F01092E6019CC087E099E099
:1057B0000E94D40781E08093E701B1C081EE98E0B8
:1057C0000E94D4078FEC98E00E94D40780911501C5
:1057D0001F928F938CEC98E09F938F930E946D089B
:1057E0008AEC98E00E94D40788EB98E00E94D407E6
:1057F000809114011F928F9385EB98E09F938F9374
:105800000E946D0883EB98E00E94D40784EA98E038
:105810000E94D407809113011F928F9381EA98E030
:105820009F938F930E946D088FE998E00E94D407A0
:105830008EE898E00E94D407809112011F928F9306
:105840008BE898E09F938F930E946D0889E898E019
:105850000E94D40784E798E00E94D4078091110148
:105860001F928F9381E798E09F938F930E946D081A
:105870008FE698E00E94D40788E598E00E94D4075C
:10588000809110011F928F9385E598E09F938F93ED
:105890000E946D0883E598E00E94D4078DB79EB7FB
:1058A00048960FB6F8949EBF0FBE8DBF1BC0CE5159
:1058B000EC2FF0E0E15DFE4F80818093E60112C0A5
:1058C00061E003C061E006C06AE08091E6010E94E9
:1058D0006F2708C08091E6010E94122803C088EF5C
:1058E00098E013C08091E601882369F01F928F939E
:1058F00082EF98E09F938F930E946D080F900F9016
:105900000F900F9004C08FEE98E00E94D40781E0C2
:1059100006C01092E70180E002C080E001CFCF9185
:105920000895E1E8F0E08081886080838081816073
:1059300080838FB7F89493E09093890090ED9093D3
:1059400088008FBF0895EFE6F0E080818260808359
:105950000895EFE6F0E080818D7F80830895EFE683
:10596000F0E0908182E08927808308951F920F9252
:105970000FB60F9211242F933F934F935F936F9322
:105980007F938F939F93AF93BF93EF93FF938091F8
:10599000E8019091E90101969093E9018093E80173
:1059A000811103C082E00E94C30DE091E901E695F8
:1059B000E695F0E0EC53F14FE4918091E8018E130D
:1059C00003C080E00E94C30DFF91EF91BF91AF91A2
:1059D0009F918F917F916F915F914F913F912F9107
:1059E0000F900FBE0F901F90189504D06894B111BE
:1059F0008DC0089570D088F09F5790F0B92F9927E7
:105A0000B751A0F0D1F0660F771F881F991F1AF0C9
:105A1000BA95C9F712C0B13081F077D0B1E00895DE
:105A200074C0672F782F8827B85F39F0B93FCCF35F
:105A3000869577956795B395D9F73EF490958095BF
:105A4000709561957F4F8F4F9F4F0895E89409C0DF
:105A500097FB3EF490958095709561957F4F8F4FA1
:105A60009F4F9923A9F0F92F96E9BB279395F695B7
:105A7000879577956795B795F111F8CFFAF4BB0F35
:105A800011F460FF1BC06F5F7F4F8F4F9F4F16C099
:105A9000882311F096E911C0772321F09EE8872F23
:105AA000762F05C0662371F096E8862F70E060E0DF
:105AB0002AF09A95660F771F881FDAF7880F969558
:105AC000879597F9089557FD9058440F551F59F041
:105AD0005F3F71F04795880F97FB991F61F09F3FDB
:105AE00079F087950895121613061406551FF2CF04
:105AF0004695F1DF08C0161617061806991FF1CF54
:105B000086957105610508940895E894BB2766277A
:105B10007727CB0197F908950BD078C069D028F08A
:105B20006ED018F0952309F05AC05FC01124EECF53
:105B3000CADFA0F3959FD1F3950F50E0551F629FE8
:105B4000F001729FBB27F00DB11D639FAA27F00DD6
:105B5000B11DAA1F649F6627B00DA11D661F829FFD
:105B60002227B00DA11D621F739FB00DA11D621FE2
:105B7000839FA00D611D221F749F3327A00D611DFF
:105B8000231F849F600D211D822F762F6A2F1124E1
:105B90009F5750408AF0E1F088234AF0EE0FFF1F34
:105BA000BB1F661F771F881F91505040A9F79E3F6B
:105BB000510570F014C0AACF5F3FECF3983EDCF3C0
:105BC000869577956795B795F795E7959F5FC1F7A8
:105BD000FE2B880F911D9695879597F9089597F953
:105BE0009F6780E870E060E008959FEF80EC089583
:105BF00000240A94161617061806090608950024AC
:105C00000A9412161306140605060895092E039425
:105C1000000C11F4882352F0BB0F40F4BF2B11F499
:105C200060FF04C06F5F7F4F8F4F9F4F0895991B98
:105C300079E004C0991F961708F0961B881F7A9583
:105C4000C9F78095089597FB072E16F4009407D0A6
:105C500077FD09D00E943D2E07FC05D03EF49095BB
:105C600081959F4F0895709561957F4F0895EE0F30
:105C7000FF1F0590F491E02D0994AA1BBB1B51E175
:105C800007C0AA1FBB1FA617B70710F0A61BB70BAC
:105C9000881F991F5A95A9F780959095BC01CD0151
:105CA0000895F999FECF92BD81BDF89A992780B5E4
:105CB0000895A8E1B0E042E050E00C94742E262F45
:105CC000F999FECF1FBA92BD81BD20BD0FB6F894E1
:105CD000FA9AF99A0FBE019608950E945F2E272F17
:105CE0000C94602EDC01CB01FC01F999FECF06C0BB
:105CF000F2BDE1BDF89A319600B40D92415050408A
:085D0000B8F70895F894FFCFF5
:105D08002002C40DB50E920E5E0E2A0E0101C501C9
:105D180028080A03140A3F4D3620394406F705C1FE
:105D280005A1056805DB04F4040D052605460501F3
:0A5D38000203040506070809000035
:00000001FF
